:100000000C9477040C9494040C9494040C9494042D
:100010000C9494040C9494040C9494040C94940400
:100020000C9494040C9494040C9494040C949404F0
:100030000C9494040C9494040C9494040C9415055E
:100040000C9494040C9494040C9494040C949404D0
:100050000C9494040C9494040C9494040C949404C0
:100060000C9494040C9494040C9494040C949404B0
:100070000C9494040C9494040C9494040C949404A0
:100080000C9494040C9494040C949404230728076F
:100090004A077907E0072C087D08C90800093309D9
:1000A00063098F09C3092A0A760AC60A030B0000EE
:1000B00000000000000000000000C3CBC0C2CDCE95
:1000C000C520CCC5CDDE00E100AE00AE003201009F
:1000D000000000D4C0C9CBDB20CCCEC4C5CBC5C981
:1000E00000FE00C700AE008C0100000000CDC0D1B2
:1000F000D2D0CEC9CAC020CCCEC4C5CBC8001B014B
:10010000E100AE005C0300000000CDC0D1D2D0CE33
:10011000C9CAC020CFD3CBDCD2C000AE00FE00AE37
:10012000002F0400000000C8CDD4CED0CCC0D6C86B
:10013000DF004601AE00C700AE0000000000CED2D6
:10014000CAD0DBD2DC005C013201C700AE00000087
:100150000000D1CED5D0C0CDC8D2DC007801460198
:10016000C700AE0000000000D1CED5D0C0CDC8D2AF
:10017000DC20CAC0CA2E2E00AE005C01C700AE0053
:1001800000000000D3C4C0CBC8D2DC009D01AE008B
:10019000E100AE000100D710C8CCDF3A00B0018CFE
:1001A00001E1005B0202000000CAC0CDC0CBDB0051
:1001B000C4019D01E10005030B000000D4C8CBDCA5
:1001C000D2D0DB00D901B001E100AE000000000098
:1001D000C7CDC0D7C5CDC8DF00EF01C401E100AE77
:1001E0000000000000C2DBD0C0C6C5CDC8DF0003E0
:1001F00002D901E100AE0000000000D3D1CBCEC295
:10020000C8DF001A02EF01E100AE0000000000D3D9
:10021000CFD0C0C2CBC5CDC8C5002E020302E100BD
:10022000AE0000000000CCC8CAD8C5D0DB00420236
:100230001A02E100AE0000000000D2C0C9CCC5D057
:10024000DB00AE002E02E100AE0000000000D1C1D4
:10025000D0CED120CCCEC4C5CBC8006E02AE009D9E
:1002600001AE0003000000CAC0CDC0CB2000820256
:100270005B029D01AE000400D40CCCC8CDC8CCD329
:10028000CC0094026E029D01AE000500D40CD6C5D0
:10029000CDD2D000A90282029D01AE000600D40C8E
:1002A000CCC0CAD1C8CCD3CC00BC0294029D01AE54
:1002B0000007000000D0C5C2C5D0D100D302A902FA
:1002C0009D01AE00080000003C2DC7C0C4C5D0C6CB
:1002D000CAC000EA02BC029D01AE0009000000C7CE
:1002E000C0C4C5D0C6CAC02D3E00AE00D3029D0119
:1002F000AE000A000000D0C0C2CDDBC520D0C0D106
:10030000D5CEC4DB001A03AE00B001AE000C000075
:1003100000D4C8CBDCD2D02020002A030503B001D2
:10032000AE000D000000D2C8CF003E031A03B0019A
:10033000AE000E000000D3D1CBCEC2C8C5004D0325
:100340002A03B001AE000F000000000000AE003E26
:1003500003B001AE00100000000000007403AE0006
:10036000FE00AE0000000000C7C2D3CA20CFD3CB2E
:10037000DCD2C0008A035C03FE00AE000000000077
:10038000CFCEC4D1C2C5D2CAC000A8037403FE0038
:10039000AE0000000000D5D0C0CDC8CBC8D9C52064
:1003A000CCCEC4C5CBC5C900C6038A03FE00AE00CF
:1003B00000000000CED0C3C0CDDB20D3CFD0C0C260
:1003C000CBC5CDC8DF00DE03A803FE00AE000000F1
:1003D0000000CACDCECFCAC820CCC5CDDE00F903FF
:1003E000C603FE00AE0000000000CFD0C5C4D3CFCE
:1003F000D0C5C6C4C5CDC8DF001304DE03FE00AE01
:100400000000000000CDC0D1D2D0CEC9CAC8205053
:10041000504D00AE00F903FE00AE0000000000D217
:10042000D0C5CDC5D0202F20D3D7C5CDC8CA00494F
:1004300004AE001B01AE0000000000C2C5D0D1C850
:10044000DF20D1C1CED0CAC800AE002F041B01AE40
:100450000000000000CE20D5D0C0CDC8CBC8D9C583
:1004600000C7CDC0D7C5CD2E22CBCEC6DC222020E2
:1004700000C7CDC0D7C5CD2E2022CBCEC6DC2220D2
:1004800000CAC0CDC0CB2022CBCEC6DC222020208B
:1004900000D4C8CAD12EC7CDC0D7C5CDC8C520206D
:1004A000202020CDC5D200CAC0CDC0CB2020202026
:1004B000202020202020202020CDC5D200C7CDC064
:1004C000D7C5CD2E22C8D1D2C8CDC02200CAC0CD3A
:1004D000C0CB2022C8D1D2C8CDC0222000CAC0CDF6
:1004E000C0CB2022C8D1D2C8CDC0222000D4C8CAD7
:1004F000D12EC7CDC0D7C5CDC8C5202000CAC0CD1C
:10050000C0CB2020202020202020202000202020C0
:10051000CDC5D2005D2D0020203C002B5B002020AB
:1005200020202020202000D3D1CB2EC7CDC0D72E15
:100530002FC7CDC0D72E00D3D1CB2ECAC0CDC0CBB4
:100540002FC7CDC0D72E00D3D1CB2ECAC0CDC0CBA4
:100550002FCAC0CDC0CB00D4C8CAD1C8D0CEC22EFD
:1005600020C7CDC0D72E00D4C8CAD1C8D0CEC22E85
:1005700020CAC0CDC0CB0020002D003E005D2D0064
:1005800020203C002B5B0020202020202020202049
:1005900000C2DBCACB00C2CACB2E00200020202024
:1005A000202020202000202020202020202000C2E9
:1005B000DBCACB00C2CACB2E002020202020202066
:1005C0002020005D2D0020203C002B5B00202020FF
:1005D00020005D2D0020203C002B5B0020202020EF
:1005E000202020005D2D0020203C002B5B002020DF
:1005F000202020002D003E005D2D0020203C002BFF
:100600005B002020202020202020200020202020EF
:1006100020003E005D2D0020203C002B5B003E00B2
:100620005D2D0020203C002B5B000000000000003E
:10063000002F00000000000300030000143E143EE1
:10064000140012257F2912001309043211001A2503
:10065000357A00000003000000000000001E2100A9
:10066000211E0000000014081400000008083E08C5
:1006700008004030000000000808080800000020C2
:10068000000000002018040300001E2525291E007C
:1006900020223F202000322929292600122121254D
:1006A0001A001814123F10002725252519001E25B1
:1006B000252518000101390503001A2525251A00F2
:1006C000062929291E00001200000000C0B2808007
:1006D00080000008142200001414141400000022EA
:1006E00014080000020129060000000000000000BC
:1006F0003C0A090A3C003F2525251A001E2121211C
:1007000012003F2121120C003F25252521003F0525
:10071000050501001E2129291A003F0404043F0099
:1007200000213F2100001020211F01003F040A1179
:1007300020003F20202020003F020C023F003F020B
:1007400004083F001E2121211E003F09090906005F
:100750001E2129313E403F0909192600122525296D
:10076000120001013F0101001F2020201F00031C77
:10077000201C03001F2018201F00310A040A31002A
:100780000304380403003129252321000000003F21
:100790002100030418200000213F00000000040293
:1007A000010204002020202020000001020000009F
:1007B0003C0A090A3C003F25252911003F25252533
:1007C0001A003F0101010100603C223F60003F250B
:1007D00025252100310A3F0A3100122121251A0066
:1007E0003F1008043F003F1009043F003F040A1176
:1007F0002000201E01013F003F0204023F003F0491
:1008000004043F001E2121211E003F0101013F0081
:100810003F09090906001E212121120001013F01A3
:100820000100132424241F001C123F121C00310A53
:10083000040A31003F2020203F60070808083F00DD
:100840003F203F203F003F203F203F60013F2424C6
:1008500018003F2438003F00003F242418001221D4
:1008600025251E003F041E211E00261909093F00F0
:10087000CCCEC4C5CBC800D1C1D0CED100C7C0C377
:10088000D0D3C7C8D2DC00C7C0CFC8D1C0D2DC002B
:10089000CAC0CDC0CB00700877087D0887089008D3
:1008A000202030252000202B2D30313233343536B6
:1008B0003738394142434445464748494A4B4C4DF5
:1008C0004E4F505152535455565758595AC1C3C49C
:1008D000C6C7C8C9CBCFD3D4D6D7D8D9DCDBDADDED
:1008E000DEDF00C3CED2CEC2CE00205B00001124DA
:1008F0001FBECFEFD0E1DEBFCDBF11E0A0E0B1E081
:10090000E2E0F3E202C005900D92A030B107D9F702
:1009100015E0A0E0B1E001C01D92A934B107E1F7F4
:100920000E9496040C947F110C9400001BBA9FEF58
:100930009ABB98BB81E887BB81E085BB8EEF84BB07
:1009400092BB11BA87EF83B988E082B91092620036
:10095000109261008FE08093650080E180936400D5
:100960000E942E110E94A00D0E940C050E949D065F
:100970008EE7809306018AE0809305010E941B1098
:1009800089ED9BE00E943111909107018091030154
:10099000981749F0909303010E94D604E09137051F
:1009A000F091380509950E94550DEECF26B32E77AC
:1009B0002E3749F410920101209302012093040183
:1009C000109200010895809100018130F1F0809132
:1009D0000201281729F010920101209302010895C5
:1009E000809101018F5F809301019091050189172A
:1009F00061F42093040110920101809106012823E3
:100A0000281719F081E08093000108958091040176
:100A10009EE79093040108958FE083BF8CE981BF26
:100A200087B7826087BF7894089578941F920F9259
:100A30000FB60F9211248F93809107018F5F8093DF
:100A400007018F910F900FBE0F901F901895809106
:100A50007A08803118F48F5F80937A080895809126
:100A60007A08833018F0815080937A080895809135
:100A70002701882319F08150809327010895409120
:100A80002701242F30E080917A0890E00197281701
:100A900039071CF44F5F409327010895E091280126
:100AA000F0912901908180913001981714F49F5F93
:100AB00090830895E0912801F0912901908180911F
:100AC0000801891714F4915090830895E09127014B
:100AD000F0E0EE0FFF1FEE0FFF1FE059F74F968576
:100AE000892F8F5F81709E7F892B86870895E09183
:100AF0002701F0E0EE0FFF1FEE0FFF1FE059F74F49
:100B00009685892F8E5F82709D7F892B86870895B9
:100B1000E0912701F0E0EE0FFF1FEE0FFF1FE059FD
:100B2000F74F9685892F8C5F8C71937E892B8687F2
:100B30000895E0912701F0E0EE0FFF1FEE0FFF1F79
:100B4000E059F74F9685892F84508C71937E892BBD
:100B500086870895E0912701F0E0EE0FFF1FEE0F6A
:100B6000FF1FE059F74F9685892F805E807E9F7129
:100B7000892B86870895E0912701F0E0EE0FFF1F93
:100B8000EE0FFF1FE059F74F9685892F8052807E28
:100B90009F71892B868708958091BB08883018F44F
:100BA0008F5F8093BB0808958091BB08833018F055
:100BB00081508093BB08089580912701882319F004
:100BC000815080932701089540912701242F30E020
:100BD0008091BB0890E00197281739071CF44F5FFC
:100BE00040932701089580912701E82FF0E0EE0F50
:100BF000FF1FE354F74F2081822F829586958770DF
:100C000090E0049734F4822F805E807E2F71822BD7
:100C10008083089580912701E82FF0E0EE0FFF1FF9
:100C2000E354F74F9081892F82958695877031F034
:100C3000892F8052807E9F71892B80830895E09157
:100C40002701F0E0EE0FFF1FE354F74F9081892F4B
:100C50008F5F8F71907E892B80830895E0912701AB
:100C6000F0E0EE0FFF1FE354F74F9081892F815082
:100C70008F71907E892B80830895E0912701F0E0A9
:100C8000EE0FFF1FE454F74F9081892F8F5F8F7015
:100C9000907F892B80830895E0912701F0E0EE0F8B
:100CA000FF1FE454F74F9081892F81508F70907F00
:100CB000892B80830895E0912701F0E0EE0FFF1F5C
:100CC000E454F74F9081892F805F807F9F70892B3C
:100CD00080830895E0912701F0E0EE0FFF1FE454B8
:100CE000F74F9081892F8051807F9F70892B80835F
:100CF000089520E08E3A920711F481E008959093D0
:100D00002C0180932B0180E0089540912B0150919C
:100D10002C0190E00BC0FA0132962591349160E0ED
:100D20002E3A360709F49A019F5FA901981798F3A4
:100D300050932C0140932B01089587EC90E0909301
:100D40002C0180932B011092090110922501109221
:100D50002A0108951F93182F813021F48BE196E02A
:100D600061E003C087E196E060E00E94930F81E0BC
:100D700090E062E0412F0E94BF0F113021F484E126
:100D800096E061E003C082E196E060E00E94930F8C
:100D90001F9108951F93182F813021F487E296E068
:100DA00061E003C083E296E060E00E94930FE0916F
:100DB0002701F0E0EE0FFF1FE454F74F808190E031
:100DC0008F709070019662E0412F0E94BF0F11302A
:100DD00021F480E296E061E003C08EE196E060E0FD
:100DE0000E94930F1F910895DF92EF92FF920F934D
:100DF0001F93CF93DF93162F92E090933305880FC4
:100E0000880F880F865F8093310580912B01909128
:100E10002C010C960E94930FE0912B01F0912C0174
:100E20003896E491F0E0E131F10508F02EC4EA5B78
:100E3000FF4FEE0FFF1F0590F491E02D099480E223
:100E4000612F0E94D30E809133058D37C0F31DC4EE
:100E50008CE096E0612F0E94930F113019F48BE51E
:100E600061E002C08CE3612F0E94D30EC0E7D8E09E
:100E70008991612F0E94D30E28E0CA37D207C1F7AB
:100E8000113019F48DE561E002C08EE3612F0E94FC
:100E9000D30EFBC382E096E0612F0E94930F1130C6
:100EA00021F48FEF95E061E003C08BEF95E0612FB7
:100EB0000E94930F80917A0890E062E0412F0E9497
:100EC000BF0F113099F488EF95E061E00E94930F15
:100ED00087E295E090932401809323018FE295E0CF
:100EE00090932F0180932E0182E044C286EF95E01B
:100EF00046C280912D01823031F410922701109268
:100F00002D0110922601113019F48BE261E002C02C
:100F10008CE3612F0E94D30E40912701242F30E0F3
:100F20008091260190E00396821793071CF44350AA
:100F3000409326019091270180912601981710F483
:100F400090932601E0907A0883E08E1520F4E090DB
:100F5000260124E0E20EF0902601D12ED09481E00B
:100F6000D82217C080E2612F0E94D30E8091270102
:100F7000F81611F0012F01C00D2D013011F40E945F
:100F8000C20E8F2D90E0019662E0402F0E94BF0FAD
:100F9000F394FE1438F380E2612F0E94D30E1130D7
:100FA00009F073CF84EF95E061E00E94930F87E32F
:100FB00095E090932401809323018FE395E018C17D
:100FC0008EEE95E0612F0E94930F113021F48BEE8D
:100FD00095E061E003C087EE95E0612F0E94930FDA
:100FE000E0912701F0E0EE0FFF1FEE0FFF1FE05929
:100FF000F74F838563E0412F0E94F10F113009F014
:1010000044CF84EE95E061E00E94930F8EE495E07A
:1010100090932401809323018AE595E090932F011A
:1010200080932E01809106018E7180930601E091DC
:101030002701F0E0EE0FFF1FEE0FFF1FCF018558D5
:10104000974F909329018093280183E880930801AA
:10105000E458F74F80814EC08CED95E0612F0E94DF
:10106000930F113021F489ED95E061E003C085ED27
:1010700095E0612F0E94930FE0912701F0E0EE0FC1
:10108000FF1FEE0FFF1FE458F74F808163E0412FF1
:101090000E94F10F113009F0F8CE82ED95E061E089
:1010A0000E94930F8EE495E0909324018093230196
:1010B0008AE595E090932F0180932E01E09127011E
:1010C000F0E0CF01880F991F880F991F8458974F20
:1010D0009093290180932801EE0FFF1FEE0FFF1F51
:1010E000DF01A059B74F1B968C9180930801EE58F1
:1010F000F74F838580933001C8C28DEC95E0612F56
:101100000E94930F113021F48AEC95E061E003C056
:1011100086EC95E0612F0E94930FE0912701F0E0AB
:10112000EE0FFF1FEE0FFF1FEE58F74F838563E0B2
:10113000412F0E94F10F113009F0A7CE83EC95E00A
:1011400061E00E94930F8EE495E0909324018093D8
:1011500023018AE595E090932F0180932E018091E1
:1011600006018E7180930601E0912701F0E0EE0FF9
:10117000FF1FEE0FFF1FCF018358974F9093290158
:1011800080932801E458F74F8081809308018DE710
:10119000B1CF89EB95E0612F0E94930F113019F4C4
:1011A0008BE261E002C08CE3612F0E94D30EE091DC
:1011B0002701F0E0EE0FFF1FEE0FFF1FE059F74F82
:1011C000868580FF03C084EB95E002C08FEA95E03E
:1011D000612F0E94930F113009F057CE8DE261E02C
:1011E0000E94D30E86E695E090932401809323011C
:1011F00090932F0180932E018EE78093060145C2C4
:1012000086EA95E0612F0E94930F113019F48BE26A
:1012100061E002C08CE3612F0E94D30EE0912701B0
:10122000F0E0EE0FFF1FEE0FFF1FE059F74F86852E
:1012300090E08C719070969587959695879561E072
:10124000412F0E94BF0F113009F01FCE8DE261E0E7
:101250000E94D30E88E895E09093240180932301A7
:1012600089E995E0C5CF8DE995E0612F0E94930F44
:10127000113019F48BE261E002C08CE3612F0E940F
:10128000D30EE0912701F0E0EE0FFF1FEE0FFF1FDE
:10129000E059F74F868582958695877090E061E0EA
:1012A000412F0E94BF0F113009F0EFCD8DE261E0B8
:1012B0000E94D30E8AEA95E0909324018093230143
:1012C0008BEB95E095CF8BE995E0612F0E94930F12
:1012D000113019F48BE261E002C08CE3612F0E94AF
:1012E000D30EE0912701F0E0EE0FFF1FEE0FFF1F7E
:1012F000E059F74F868581FF03C086E995E002C07B
:1013000081E995E0612F0E94930F113009F0BDCD66
:101310008DE261E00E94D30E87E795E065CF87E814
:1013200095E0612F0E94930F113021F484E895E03D
:1013300061E003C080E895E0612F0E94930F8091E7
:10134000BB0890E061E0412F0E94BF0F1130A9F46B
:101350008DE795E061E00E94930F8CEC95E090930F
:1013600024018093230184ED95E090932F018093D5
:101370002E018BE080932D0188C18BE795E0612FD2
:101380000E94930F82C180912D018B3031F4109215
:10139000270110922D0110922601113019F48BE2D1
:1013A00061E002C08CE3612F0E94D30E40912701BF
:1013B000242F30E08091260190E004968217930755
:1013C0001CF44450409326019091270180912601FE
:1013D000981710F490932601E090BB0824E02E1596
:1013E00020F4E090260185E0E80EF0902601D12E51
:1013F000D09421E0D22217C080E2612F0E94D30E48
:1014000080912701F81611F0012F01C00D2D013038
:1014100011F40E94C20E8F2D90E0019661E0402FE2
:101420000E94BF0FF394FE1438F380E2612F0E94F4
:10143000D30E113009F029CD89E795E061E00E94D3
:10144000930F8CED95E0909324018093230184EE1B
:1014500095E0CECE87E795E0612F0E94930F113083
:1014600019F48BE261E002C08CE3612F0E94D30E7D
:10147000E0912701F0E0EE0FFF1FE354F74F80816A
:1014800082958695877090E082309105A1F0833037
:1014900091052CF4009749F00197C1F409C08330FD
:1014A000910561F0049791F40CC087E695E00BC0BC
:1014B00087E595E008C087E495E005C087E395E0FF
:1014C00002C087E295E0612F0E94930F113009F06E
:1014D000DCCC8DE261E00E94D30E83EF95E0909327
:1014E0002401809323018AE096E0CBC08EE195E051
:1014F000612F0E94930FE0912701F0E0EE0FFF1F94
:10150000E354F74F808182958695877090E002972B
:1015100064F1113021F48BE195E061E003C087E1D3
:1015200095E0612F0E94930FE0912701F0E0EE0F0C
:10153000FF1FE354F74F808190E08F719070019608
:1015400062E0412F0E94BF0F113009F09ECC84E170
:1015500095E061E00E94930F8FE196E09093240163
:10156000809323018EE296E08CC08DE095E0612FA0
:101570000E94930F113009F088C01092240110923C
:10158000230110922F0110922E017FC0E0912701BC
:10159000F0E0EE0FFF1FE354F74F808182958695B0
:1015A000877090E082309105A1F0833091052CF492
:1015B000009749F00197C1F409C08330910561F0AB
:1015C000049791F40CC08DEF94E00BC08DEE94E085
:1015D00008C08DED94E005C08DEC94E002C08DEB69
:1015E00094E0612F0E94930F812F0E94CA06113050
:1015F00009F04BC08DE396E0909324018093230182
:101600008CE496E03EC0E0912701F0E0EE0FFF1F72
:10161000E354F74F808182958695877090E0823001
:101620009105B9F0833091052CF4009749F00197AA
:10163000F1F409C08330910579F00497C1F40FC02B
:1016400087EA94E002C081E994E0612F0E94930F41
:101650000EC081E894E005C081E794E002C081E615
:1016600094E0612F0E94930F812F0E94AA061130EF
:1016700061F48BE596E090932401809323018AE640
:1016800096E090932F0180932E01E0912B01F09131
:101690002C018591949120E08E3A920711F481E01B
:1016A00005C090932C0180932B0180E0DF91CF91B6
:1016B0001F910F91FF90EF90DF9008950F93CF93BC
:1016C000DF9381E080933205109224011092230170
:1016D00010922F0110922E010E948A0DC0912B01B1
:1016E000D0912C0180E063E043E023E001E00E9420
:1016F000150EE0912B01F0912C0134968591949177
:1017000090932C0180932B0124E0209333051092B9
:1017100031050C9660E00E94930F809133058F5F36
:1017200063E04FE723E00E94150E80E063E040E0B5
:101730002CE30E94150E8FE763E04FE72CE30E9435
:10174000150E80E06CE34FE72CE30E94150ED0935A
:101750002C01C0932B01809109010E94850600E0B5
:1017600009C0802F60E00E94F406813011F40091DE
:1017700009010F5F80910901081798F3802F61E03C
:101780000E94F406813089F00091090107C0802F82
:1017900060E00E94F406813009F406E00F5F063035
:1017A000B0F3D0932C01C0932B01DF91CF910F9117
:1017B000089580914805882329F40E945E0B81E0FA
:1017C000809348050E9406058E3709F4ECC08637E1
:1017D00009F463C0873748F48E3509F44CC08E365F
:1017E00059F08E3309F0DDC037C08A3709F4B4C030
:1017F0008C3709F0D6C090C080910901882319F078
:1018000081508093090120912B0130912C01F90125
:1018100032968591949140E08E3A940729F0909306
:101820002C0180932B01BDC040E0F901859194917A
:10183000542F5F5F60E08E3A960719F09C01452FA8
:10184000F4CF4093090130932C0120932B014630B3
:1018500008F4A7C085E03EC0209123013091240107
:101860002115310509F49DC0E0912B01F0912C0167
:101870003996E4910EC020912E0130912F0121154F
:10188000310509F48EC0E0912B01F0912C013996BD
:10189000E4918E2FF901099584C080912B019091DC
:1018A0002C01FC0125913491E0E02E3A3E0749F0ED
:1018B00030932C0120932B0180910901853048F051
:1018C00070C0FC013496859194918217930729F496
:1018D00011C08F5F8093090164C090932C018093A5
:1018E0002B01FC01369685919491F0E08E3A9F078A
:1018F00071F425C087EC90E090932C0180932B012C
:10190000109209011092250110922A014AC0909369
:101910002C0180932B0113C01092480540912B019C
:1019200050912C01CA010696FC0125913491F0E0FA
:101930002E3A3F0739F030932C0120932B0110925F
:1019400009012FC0465F5F4FFA018591949100977E
:1019500041F10E94311125C080912501882309F5AC
:10196000E0912B01F0912C0134964591549120E0A7
:101970004E3A5207B1F0CA0120E00BC0FC0132968A
:1019800085919491322F3F5F60E08E3A960719F06F
:10199000232F253098F32093090150932C01409375
:1019A0002B010E945E0B08950F931F93E0912B0172
:1019B000F0912C01389684918530D1F08630E9F190
:1019C000843009F058C08091270190E0880F991F5A
:1019D000880F991FFC01E458F74FE081DC01ED39D5
:1019E00024F0A059B74F8CE93DC0A059B74F41C072
:1019F000E0912701F0E08F01000F111F000F111F70
:101A00000458174FEE0FFF1FEE0FFF1FDF01AE58F8
:101A1000B74F1B968C91992787FD9095E059F74F0A
:101A20002385332727FD3095820F931F62E070E0F6
:101A30000E946C11F80160831EC08091270190E024
:101A4000FC01EE0FFF1FEE0FFF1FE458F74FE08180
:101A5000DC01AA0FBB1FE43644F4AA0FBB1FAE582B
:101A6000B74F84E61B968C9306C0AA0FBB1FAE58D7
:101A7000B74F1B96EC930E9445111F910F9108954B
:101A800095B3957E95BB9FEF9ABB8BBBAD9AAD98F6
:101A9000A99A089595B39D7E95BBAB9A9FEF9ABB8B
:101AA0008BBBAD9AAD98A99A0895EF92FF920F93D0
:101AB0001F93CF93DF9380913205813021F500E0B1
:101AC000C0E0D0E0802F806B0E94400D80E10E943A
:101AD000400D84E00E94400D10E081E3E82E81E09B
:101AE000F82EEC0EFD1EF701E10FF11D80810E9422
:101AF0004A0D1F5F1038B9F70F5FC058DF4F08302D
:101B000009F710923205DF91CF911F910F91FF904D
:101B1000EF90089580E090E00DC0FA01E20FF11D12
:101B200010822F5F2038C9F780589F4F24E0803003
:101B3000920729F020E0AC014F5C5E4FEECF089594
:101B400085B3847085BB85E0982F9A95F1F78A95C7
:101B5000F1F7AA9A80E797E10197F1F782EE0E94E8
:101B6000400D8EEA0E94400D81EA0E94400D86EAF7
:101B70000E94400D84EA0E94400D82EA0E94400DBE
:101B800080EC0E94400D8FE20E94400D85E20E9491
:101B9000400D81E80E94400D82E20E94400D8FEAD4
:101BA0000E94400D0E948A0D0E94550D08951F93BA
:101BB000182F81E80E94400D812F0E94400D1F9137
:101BC0000895782F87FD30C0603470F5262F277078
:101BD00081E090E0582F01C0550F2A95EAF76695ED
:101BE00066956695262F30E0872F90E0442371F0AC
:101BF000F901F695FE2FEE27F795E795E80FF91F07
:101C0000EF5CFE4F8081852B80830895F901F69566
:101C1000FE2FEE27F795E795E80FF91FEF5CFE4FD3
:101C2000509580815823508308956F927F928F92B0
:101C30009F92AF92BF92CF92DF92EF92FF920F935B
:101C40001F93CF93DF93C82ED62E602E042F081B30
:101C5000122F161B712E07FD03C08824839404C025
:101C6000082F041B88248A9417FD03C09924939499
:101C700004C01D2D121B99249A94011738F4FD2CD1
:101C8000E12EAD2CBB24C02FD0E045C0FC2CE02EB3
:101C9000AC2CBB24C12FD0E01DC02F2D30E0171479
:101CA0001CF42A193B0904C0C501821B930B9C013B
:101CB0002C9FC0012D9F900D3C9F900D1124602FF3
:101CC00070E00E946C116D0D8F2D462D0E94E10D6C
:101CD000F80CEA94EE2009F720C02F2D30E01714FD
:101CE0001CF42A193B0904C0C501821B930B9C01FB
:101CF0002C9FC0012D9F900D3C9F900D1124612FB2
:101D000070E00E946C116C0D862F6F2D462D0E9485
:101D1000E10DF90CEA94EE2001F7DF91CF911F91CC
:101D20000F91FF90EF90DF90CF90BF90AF909F907A
:101D30008F907F906F900895CF92DF92EF92FF92F5
:101D40000F931F93182FF62EE42ED22E2F2D0E94C4
:101D5000150E812F6D2D4E2D2D2D0E94150E812FCC
:101D60006F2D412F2D2D0E94150E8E2D6F2D4E2D76
:101D70002D2D0E94150E1F910F91FF90EF90DF9077
:101D8000CF9008951F9310E0809133056091310545
:101D90006150610F815041E00E94E10D1F5F1830DA
:101DA00099F71F9108956F927F928F929F92AF92B1
:101DB000BF92CF92DF92EF92FF920F931F93CF9338
:101DC000DF93A62E8F3728F4482F40522AE236E0C0
:101DD00004C0482F405C20EB37E082E0A81611F4E5
:101DE000A090340580913105082F009507708695E5
:101DF0008695869590E03C017694762C66247794BF
:101E000067946C010894C11CD11CD694DC2CCC24A2
:101E1000D794C79486E0489FE0011124C20FD31FD6
:101E2000BB24802F90E047E0E42EF12CE81AF90A59
:101E30004C010894811C911CFE018491AA2011F48C
:101E4000182F0CC0182F109560913105662331F0C2
:101E500061508091330541E00E94E10D909133057E
:101E6000692F70E0F301E60FF71F1F77412F50E055
:101E7000EF5CFE4F9A010E2C02C0220F331F0A9412
:101E8000E2F78081820F8083073071F0F601E60F60
:101E9000F71FEF5CFE4F082C02C0559547950A943A
:101EA000E2F78081840F8083892F8F5F80933305D1
:101EB0008F3730F4B3942196F6E0BF1609F0BCCF0B
:101EC000DF91CF911F910F91FF90EF90DF90CF9016
:101ED000BF90AF909F908F907F906F9008951F93C9
:101EE000CF93DF93162FE82FF0E0EE0FFF1FEA5697
:101EF000F74FC591D49104C0612F0E94D30E219653
:101F0000FE0184918823C1F7DF91CF911F9108953D
:101F1000982F84568C3518F40E946F0F0895892FDE
:101F20000E94D30E08950F931F93CF93DF93EC017C
:101F3000062F623011F4009134050130B9F480911C
:101F40003305882399F010E08091330560913105C5
:101F50006150610F815041E00E94E10D1F5F183018
:101F600099F704C0602F0E94880F2196FE0184918A
:101F70008823C1F7DF91CF911F910F910895DF92D0
:101F8000EF92FF920F931F93CF93DF93F82E092FB9
:101F9000D62EE42EC0E1D7E215E0D11650F08F2DF9
:101FA000902FBE010E945811862F805D6E2D0E94D9
:101FB000D30E115071F08F2D902FBE010E94581139
:101FC000F82E092FCE016AE070E00E945811EB0153
:101FD000E4CFDF91CF911F910F91FF90EF90DF90B1
:101FE0000895FF920F931F93182FF62E042F882326
:101FF00031F480EA98E0642F0E94930F18C087FFA5
:1020000006C08DE2642F0E94D30E119504C08BE2AE
:10201000642F0E94D30E812F992787FD90956F2DF5
:10202000402F0E94BF0F85E2602F0E94D30E1F91A8
:102030000F91FF9008958CEC809370088EEC809344
:10204000710884EC8093720885EC809373088BECA4
:10205000809374088CED8093750880E280937608F5
:1020600080ED8093770883ED8093780881ED8093ED
:10207000790888E080937A08EBE7F8E02CE994E6A9
:1020800082E02083118292838383349638E0EB3B95
:10209000F307B9F788E0819380E0808311828F5F36
:1020A00032968830D1F70895CF92DF92EF92FF9267
:1020B0000F931F93CF93DF9311E0109332050E948B
:1020C0008A0D8EE0809333051093310588E991E005
:1020D00060E00E94930F8AEE98E060E00E94930F08
:1020E000C0E7D8E010E080913605181711F060E0E5
:1020F00003C00E94C20E61E089910E94D30E1F5F4F
:102100001A3089F78DE560E00E94D30E9CE0C92E5D
:10211000EE24FF24C0923105E701CA55D74F87014D
:1021200087E0D82ED09233058091350590E0801756
:10213000910711F060E003C00E94C20E61E0FE0151
:1021400084910E94D30EFAE0DF0E0F5F1F4F21969D
:102150008FE7D81639F798E0C90EECE0F0E0EE0E04
:10216000FF1EF4E3CF16B1F68EE28093330585E3CC
:1021700080933105809135058C3310F460E003C005
:102180000E94C20E61E083EE98E00E94930F84E00B
:1021900069E04CE72DE301E00E949C0EDF91CF91B6
:1021A0001F910F91FF90EF90DF90CF900895809155
:1021B0004805882349F4109236051092350581E0D0
:1021C000809348050E9454100E9406058E3709F43A
:1021D00044C08E3661F08F3628F48E33B1F08E35E0
:1021E000D1F519C0863749F08C37A9F51AC080910E
:1021F00035058C3080F18C5005C0809135058C33CD
:1022000050F5845F8093350526C08091350588237D
:1022100011F18150F7CF809135058C33E0F48F5F59
:10222000F1CF909135059C33A0F480913605E92FCC
:10223000F0E0EA55F74F9491E82FF0E0E059F74FBE
:1022400090838F5F809336058A3029F4109236058B
:1022500002C00E9445110E94541008951092470533
:10226000089520914705E22FF0E0EE0FFF1FE75C95
:10227000FA4F918380832F5F209347059093380511
:1022800080933705109248050895E0914705E15085
:10229000E0934705F0E0EE0FFF1FE95CFA4F808105
:1022A00091819093380580933705109248050895E1
:1022B000AA1BBB1B51E107C0AA1FBB1FA617B7076C
:1022C00010F0A61BB70B881F991F5A95A9F7809588
:1022D0009095BC01CD01089597FB092E07260AD0E1
:1022E00077FD04D0E5DF06D000201AF470956195E3
:1022F0007F4F0895F6F7909581959F4F0895F89434
:02230000FFCF0D
:00000001FF
